:020000040800F2
:1000000000800030212500086F1100086F110008E2
:100010006F1100086F1100086F1100080000000048
:100020000000000000000000000000007111000846
:10003000711100080000000071110008A9180008E3
:100040006F1100086F1100086F1100086F11000890
:100050006F1100086F1100086F1100086F11000880
:100060006F1100086F1100086F110008B91800081F
:100070006F1100086F1100086F1100086F11000860
:100080006F1100086F1100086F1100086F11000850
:100090006F1100086F1100086F1100086F11000840
:1000A0006F1100086F1100086F1100086F11000830
:1000B0006F1100086F1100086F1100086F11000820
:1000C0006F1100086F1100086F1100086F11000810
:1000D0006F1100086F1100086F1100086F11000800
:1000E0006F1100086F110008000000006F11000878
:1000F0006F1100086F1100086F1100086F110008E0
:100100006F1100086F1100086F1100086F110008CF
:100110006F1100086F1100086F1100086F110008BF
:100120006F1100086F1100086F1100086F110008AF
:100130006F1100086F1100086F1100086F1100089F
:1001400000000000000000000000000000000000AF
:100150006F1100086F1100086F1100086F1100087F
:100160006F1100086F1100086F1100086F1100086F
:100170006F1100086F1100086F11000800000000E7
:100180006F1100086F1100086F1100086F1100084F
:10019000731100086F1100086F1100086F1100083B
:1001A0006F1100086F1100086F11000800000000B7
:1001B0006F1100086F1100086F1100086F1100081F
:1001C0006F1100086F11000800000000000000001F
:1001D00000000000000000006F1100080000000097
:1001E000000000000000000000000000000000000F
:1001F00000000000000000006F1100086F110008EF
:100200006F1100086F110008000000006F11000856
:100210006F1100086F1100086F1100086F110008BE
:100220006F110008000000006F11000800000000BE
:100230006F1100086F110008000000006F11000826
:100240006F1100086F1100086F1100086F1100088E
:100250006F1100086F1100086F1100086F1100087E
:100260006F1100086F1100086F1100086F1100086E
:100270006F1100086F1100086F11000800000000E6
:100280006F1100086F1100086F1100086F1100084E
:10029000000000006F1100086F110008000000004E
:1002A000000000006F1100086F1100086F110008B6
:1002B0006F1100086F1100086F1100086F1100081E
:0C02C0006F1100086F1100086F1100089A
:1002CC002DE9F04FB3B040F200044FF4C020C3F25C
:1002DC00000443F200461421C4F20106A060082079
:1002EC00E06004F11C004FF4800B0025C4E9006BA6
:1002FC00C4E904554FF00058C4F8188000F08AFE89
:10030C004FF08040606304F13800242100F082FE3D
:10031C0094F88100002840F045810AA8902184F8C7
:10032C00805000F077FE0320029028200227CDE9B0
:10033C0003070B204FF40058CDE90507C0200995A1
:10034C00CDE907054FF4803018906846CDE900855B
:10035C0000F03CFA002840F0B28144F2E04040F258
:10036C000809C5F60200C4F20209016941F4005102
:10037C000161016901F400512E912E99016841F03F
:10038C001001016000682EA900F010002E902E982C
:10039C004FF4B040CDE92E070520329041F2000019
:1003AC00C5F60200CDE9305501F0D2FF40F28803CA
:1003BC005421C3F20003CC4659604021C3E9021515
:1003CC004FF4806119614FF400615D62C3E9051857
:1003DC0040F22411C3F20001C3E907550A6883F8FF
:1003EC0035705CF8087FC3F800C083F8345027F0F0
:1003FC000107CCF80070D9F808C05FEACC7C0AD0B1
:10040C00D1F800C0ACEB020CBCF1050FF3D94FF0E6
:10041C00030E20225AE048F23F02D9F80810CFF61A
:10042C00106201EA020BD3E9037547EA0B07D3E923
:10043C00018BD3E905CE3D43D3E907104CEA050CFB
:10044C005F6A41EA0C01D3E90BA20843042F42EA8C
:10045C000A0208BF1043A8F13F0140EA0B00132920
:10046C0040EA0E0507D80120884040F20F31C0F257
:10047C000F01084204D1A8F12900062880F012814E
:10048C0045F48015C9F80850042FD9F81C0020F049
:10049C00070047EA00072BD19D6A2F43BAF1000FE2
:1004AC0026D0BEF5005F08D0BEF1000F18D1022D8A
:1004BC0019D0012D0ED0B5B11AE0032D18D84FF07C
:1004CC00010E4022DFE805F0020F02065A6583F8A0
:1004DC0035E072B6AAF1C070B0FA80F0420904E0BF
:1004EC00032D40F0E680CAF30062002A40F0E3805E
:1004FC0040F6800206F54C40C4F20202C9F81C70AA
:10050C004FF0000CC3E9160C3F200127BBF1800F04
:10051C00C9F8000009F5FF60C3E918029F6605D110
:10052C00C3F804C0C9F8F8C7576019E0A8F1010076
:10053C005FFA88FC0728C9F8F8C7576010D8ACF1E7
:10054C00010CBCF1080F10D202EB8800C03200F194
:10055C007C0107FA0CFCC3E91B12C3F874C008E059
:10056C0000205867C3E91B0007E003F16C0191E818
:10057C00061000200860C2F804C04EF60C515865F5
:10058C00CEF2000183F83570A1F60442A3679C6398
:10059C00096882F84C034FF480101060D4E9006BAA
:1005AC00D4F81880022084F881003068B8F1806F8C
:1005BC0020F001003060B06800F4F81E10D1BBF1DF
:1005CC00000F05D0BBF5800F0AD1A16B69B903E010
:1005DC00A16BB1F1805F06D1316841F4805131607B
:1005EC005FEA4B2101D401230CE0E2680023072AC7
:1005FC0008D33168D4F850C021F4807141EA0C0161
:10060C00316004E0326822F480723260E268E069A2
:10061C0042EA0E02A76A1043E26B3843D4F808C0D2
:10062C001043D4E90451B060D4E90D09626A104357
:10063C00226A40EA090028430843A16DD4E912A7B5
:10064C001043384340EA0C0040EA0A000843BBF16F
:10065C00000F40EA080040EA0B00F0600BD0306D50
:10066C0020F001003065A3B9F068616D20F0004006
:10067C000843F0600DE0B068012161F3CC20B0605C
:10068C00B068022161F34A20B060306D20F00100A7
:10069C0030650020C4F88400012084F8810033B058
:1006AC00BDE8F08F28F00300742808BF45F48015CE
:1006BC00E8E6BFF41DAF4FF0010E402206E772B61C
:1006CC0044F20041C5F602010869C0F3C2000328D8
:1006DC0014D002280DD090BB0868800649F20000A7
:1006EC00C0F2D03058BF70470968C1F3C101C8408F
:1006FC00704747F64000C0F27D1070478A6A886ADE
:10070C00C0F3051CC86ABCF1000F4B6B04BF002082
:10071C00704700F0010002F003024042022A00EA96
:10072C00D3006FF35F3000EE100AB8EE400A0BD026
:10073C006AB9086880060DD49FED221A17E040F6BE
:10074C000010C0F23D0070479FED1D1A0FE09FEDA9
:10075C001B1A0CE0086849F20002C0F2D032C0F358
:10076C00C10022FA00F001EE100AB8EE411A086B33
:10077C009FED153A6FF35F2002EE100A086BC0F381
:10078C004620B8EE422A013000EE032A00EE10CAD1
:10079C00B7EE003AB8EE400A81EE000A32EE031AC8
:1007AC0020EE010A01EE100AB8EE411A80EE010AA1
:1007BC00BCEEC00A10EE100A704700BF0024744A49
:0C07CC0020BCBE4B0024744C000000391F
:1007D8002DE9F8430446C07844F210460007C5F6F0
:1007E800020621D5606E4FEA3051032931D8DFE87F
:1007F80001F002070D16F16941F40031F1610EE0D4
:1008080004F10800022101F0C5FB04E004F128000E
:10081800022101F03FFC5FEA000807D1606E316CED
:1008280021F44011084330644FF000086078C00795
:1008380001D1454624E0A06D042835D84546DFE8B7
:1008480000F003110B171700F06940F40030F06155
:100858000EE04FF00108E9E704F12800002101F05B
:1008680019FC04E004F10800002101F093FB05469F
:100878002F4635B9306CA16D20F00700084330646D
:100888004746607840072AD5D4F8A4004FEA70504C
:10089800052812D8DFE800F003140B1A1A1AF069B9
:1008A80040F40030F06111E001250127E9E704F187
:1008B8002800002101F0EEFB07E00125A8460FE023
:1008C80004F10800002101F065FB0546A8463DB982
:1008D800B06CD4F8A41020F460000843B064B846A3
:1008E8006078000727D5D4F8A8004FEA30600528BB
:1008F8000FD8DFE800F0031108171717F06940F464
:100908000030F0610EE004F12800002101F0C2FB84
:1009180007E0012501270FE004F10800002101F09C
:1009280039FB05462F463DB9B06CD4F8A81020F025
:10093800E0600843B0644746E07880071BD5E06C68
:100948004FEA3010032829D8DFE800F00D02070D20
:10095800F06940F40030F06105E004F1080002217C
:1009680001F018FB0546A84635B9F06BE16C20F09C
:1009780030000843F063B8466078C00625D5E06DBE
:100988004FEA3030042835D8DFE800F003110B17A0
:100998001700F06940F40030F0610EE00125A84628
:1009A800EAE704F12800002101F074FB04E004F1F7
:1009B8000800002101F0EEFA05462F4635B9306CE3
:1009C800E16D20F4E04008433064474660788006D3
:1009D80021D5206E4FEA3040052800F2FB82DFE87F
:1009E80000F012030C12121204F10800012101F0A8
:1009F800D1FA07E001250127E8E704F128000121E1
:100A080001F048FB0546A84635B9306C216E20F444
:100A1800E02008433064B8466078400620D5D4F812
:100A2800AC004FEA3070052800F2D782DFE800F00A
:100A38000F03090F0F0F04F10800012101F0AAFAB2
:100A480004E004F12800012101F024FB05462F46AB
:100A58003DB9B06CD4F8AC1020F0E0400843B06465
:100A68004746607800061AD5E06E80B1B0F1005FA5
:100A780007D0B0F1805F22D1F06940F40030F06116
:100A880005E004F10800012101F084FA0546A846B2
:100A980035B9306CE16E20F0405008433064B846F8
:100AA800E078C0071CD0A06C03284BD8DFE800F022
:100AB80010020A10F06940F40030F06108E00125E6
:100AC800A846EDE704F10800022101F063FA0546A3
:100AD800294635B9F06BA16C20F003000843F06398
:100AE8004146D4E90002420201D4884617E0D6F80C
:100AF800F02342F48072C6F8F02340F22412C3F2C5
:100B080000021368D6F8F073FF0506D41768FF1AB9
:100B1800642FF7D90325A84601E0A846ADB1C00760
:100B280062D0A06F4FEAF000052800F25982DFE892
:100B380000F053034D53535304F10800012101F011
:100B480029FA48E001250121CBE7336ED4F8B0C07B
:100B580083EA0C0313F4407F0BD0336E376E47F4EF
:100B680080373766376E23F4407327F4803737664B
:100B78003366BCF5807F11D1176841F288330325AD
:100B8800D6F860805FEA887808D4D2F80080A8EBAD
:100B9800070898454FF00308F2D9C0E733684FF6C5
:100BA800CF770CF4407223F47C53C0F2FF0707EAB6
:100BB8001C170025B2F5407F08BF3B4333606FF335
:100BC8001F3C326E42EA0C0232668EE704F12800BE
:100BD800012101F05FFA05462F4635B9706CA16F07
:100BE80020F03800084370644746207880071CD5F9
:100BF800606F052800F2F781DFE800F00F03090FA6
:100C08000F0F04F10800012101F0C4F904E004F118
:100C18002800012101F03EFA0546A84635B9706C56
:100C2800616F20F0070008437064B84620784007D9
:100C38001ED5D4F89000052800F2D881DFE800F02E
:100C48000F03090F0F0F04F10800012101F0A2F9A9
:100C580004E004F12800012101F01CFA0546A94628
:100C68003DB9B06CD4F8901020F007000843B06488
:100C7800C1462078800620D5D4F88C004FEA307021
:100C8800052800F2B681DFE800F00F03090F0F0F07
:100C980004F10800002101F07DF904E004F12800C6
:100CA800022101F0F7F905462F463DB9706CD4F8DA
:100CB8008C1020F0E040084370644F4620784006CE
:100CC80020D5D4F898004FEAB020052800F2948186
:100CD800DFE800F00F03090F0F0F04F108000021EF
:100CE80001F058F904E004F12800022101F0D2F9DA
:100CF8000546A8463DB9B06CD4F8981020F4E050E9
:100D08000843B064B8462078000620D5D4F89C0083
:100D18004FEA7030052800F27281DFE800F00F0317
:100D2800090F0F0F04F10800002101F033F904E066
:100D380004F12800022101F0ADF905462F463DB91E
:100D4800B06CD4F89C1020F460400843B064474667
:100D5800D4E90001010715D5D4F88000B0F5805F0B
:100D680009D104F12800022101F094F9002818BFE4
:100D78000127D4F88000716C21F440510843706455
:100D8800D4E90001C10615D5D4F89400B0F5807FE8
:100D980009D104F12800022101F07CF9002818BFCC
:100DA8000127D4F89400B16C21F440710843B06471
:100DB800D4E9000100031FD5D4F8A000B0F5003F26
:100DC80011D0B0F5803F08D0002840F0FB8004F136
:100DD8000800002101F0DEF804E004F128000221F7
:100DE80001F058F90546A8463DB9B06CD4F8A010F2
:100DF80020F440300843B064B846A07840071FD5B7
:100E0800D4F88400B0F5401F11D0B0F5001F08D009
:100E1800B0F5801F40F0D980F06940F40030F061EF
:100E280005E004F12800012101F034F905462F46B8
:100E38003DB9706CD4F8841020F4401008437064F5
:100E48004746A078C00701D1B8461AE0206DB0F532
:100E5800803F05D098B9F06940F40030F06105E0B2
:100E680004F10800022101F095F80546A84645B9A5
:100E7800F06B216D20F480300843F063E4E701252E
:100E8800A846D4E900108A000AD504F128000221F6
:100E980001F000F9002818BF4FF00108D4E900104C
:100EA8008A0316D5E26F6FF0010303EB3223022B9E
:100EB80009D34FEA322333B1012B40F08980F3691B
:100EC80043F40033F3612DB9736C23F440731A4370
:100ED80072644546CA0205D5226F336C23F000437D
:100EE8001A4332648A0205D5A26E336C23F08073EC
:100EF8001A4332644A0008D5326822F4004232604C
:100F0800D4F8B42033681A433260CA0F05D0626D32
:100F1800F36B23F040531A43F263090206D5D4F861
:100F28008810726C22F4400211437164C10709D021
:100F380004F10800002101F02DF8002818BF05462B
:100F4800D4E90010810709D504F10800012101F056
:100F580021F8002818BF0546D4E90010410709D533
:100F680004F10800022101F015F8002818BF054611
:100F7800D4E90010010709D504F12800002101F087
:100F880089F8002818BF0546D4E90010C10609D51C
:100F980004F12800012101F07DF8002818BF05465A
:100FA800D4E90010800607D504F12800022101F0D9
:100FB80071F8002818BF0125002D18BF0125284603
:100FC800BDE8F8830125A84617E70125012738E77A
:100FD80001257FE70125A8461EE50125012740E5F3
:100FE8000125012701E60125A8461FE60125A94696
:100FF8003FE60125012761E60125A84683E601258C
:041008000127A5E631
:10100C00034C206804348047FBE700F037F8FEE718
:04101C00482500085B
:1010200000220B0011001A0084465AB3830704D033
:1010300000F8011B013AF9D124E0C9B241EA0121CB
:1010400041EA0141202A11D3203A2DE9F0030B4651
:101050000C460D460E460F4688468946A0E8FA0320
:10106000203AFBD2BDE8F00320320BD0042A05D38E
:1010700040F8041B043A05D0042AF9D200F8011BF9
:08108000013AFBD16046704704
:101088004EF61450BFF35F8FCEF20000016921F4D1
:10109800803101610021C0F88010C0F88410D0F8B8
:1010A8008C2022F00102C0F88C2048F23F72C0F870
:1010B8008810C1F20402C0F88C200522C0F88020F4
:1010C800026942F480320261BFF34F8FBFF36F8F22
:1010D8000268920311D4BFF34F8FBFF36F8FC0F82C
:1010E8003C12BFF34F8FBFF36F8F016841F400319B
:1010F8000160BFF34F8FBFF36F8F0168C90326D418
:1011080000210167BFF34F8F43F6E07EC26E4FEABE
:10111800D20CC2F34E31C2F3C90301334A0102EAC9
:101128000E041D4604EB8C74013DC0F84C4204F1DA
:101138004044F9D1203A0139F1D2BFF34F8F016809
:1011480041F480310160BFF34F8FBFF36F8F00F020
:101158009AF900F019FA00F0C7FD00F0A3FD00F0BD
:0611680059FEFFF7AFF88D
:02116E00FEE79A
:021170007047C6
:1011720038B540F20004C3F20004206802694369F2
:10118200816894F881501D0507D512F008051FBF2C
:10119200816941F40061816138BD03EA020505F00D
:1011A2006402042A04D1616F20468847216F10E04F
:1011B20005F04502012A07D1216F2046884705F034
:1011C2002200022804D038BD05F02602022A04D1EA
:1011D200616F2046BDE8384008472A076BD415F4F2
:1011E200587FF0D06A0609D5D4F8842042F0040270
:1011F200C4F88420826942F040028261AA0509D5BE
:10120200D4F8842042F00102C4F88420826942F4B6
:1012120000728261EA0509D5D4F8842042F00802FE
:10122200C4F88420826942F480728261AA0609D5D8
:10123200D4F8842042F08002C4F88420826942F00B
:1012420020028261D4F88420002ABCD0026801F412
:10125200404122F001020260026940F26B33B1F5B3
:10126200404F22EA0301016140F0B980816842F2F5
:10127200493521F440418160E06FC0F6000550B16C
:10128200056500F08AFF00281EBFD4F8840040F0F4
:101292004000C4F88400A06F002894D0056500F0D7
:1012A2007CFF002808BF38BDD4F8840040F040001D
:1012B200C4F8840038BD816941F008018161816907
:1012C20041F010018161816941F40061816101692C
:1012D20021F008010161816811F4404F24D1B4F872
:1012E2006A1009B3E168102905D32268616E126B96
:1012F20041F8042B0DE0082904D3028E616E21F817
:10130200022B06E0216891F83010626E1170616E56
:1013120001316166B4F86A100139A4F86A10B4F8B0
:101322006A100029DED120684169826942F0080210
:101332008261826940F26F3342F010028261026878
:1013420022F00102026002699A430261826822F479
:101352004042826094F88120042A18BF11F02002D2
:1013620009D0D4F8842042F08002C4F88420826933
:1013720042F02002826194F88120032A18BF11F002
:10138200400209D0D4F8842042F00402C4F8842038
:10139200826942F0400282618A0509D5D4F884202C
:1013A20042F00102C4F88420826942F40072826130
:1013B200C90509D5D4F8841041F00801C4F8841095
:1013C200816941F4807181610020A4F86200A4F86F
:1013D2006A00012084F88100D4F8840038BD01201D
:0613E20084F8810038BD13
:1013E8004EF6885042F20003CEF20000C5F2002308
:1013F800026842F470020260186800F00F000628C4
:1014080004D81868072262F30300186044F2004009
:101418004EF67F51C5F60200CEF6F621026842F07C
:101428000102026000220261D0F800C001EA0C014A
:1014380001601968090705D519684FF0070C6CF3A6
:101448000301196040F200218261C0F20221C261E9
:10145800026281620021C0F2FF11C16240F2802164
:10146800C0F20111016342638163C2630164426493
:10147800016821F480210160026603F5005043F2FF
:06148800D2010160704773
:10148E0010B582B04EF60C504FF6FF02CEF20000B1
:10149E0044F21844C5F602040168114040F20032CD
:1014AE00C0F2FA5211430160FFF709F9216842F2C6
:1014BE003852C0F60002C1F30321515C226801F0DC
:1014CE001F01C84040F22C11C3F2000108600F202A
:1014DE0000F00FF858B9D4F8DC0040F00200C4F860
:1014EE00DC00D4F8DC0000F002000190019802B09C
:0214FE0010BD1F
:1015000010B540F22C1144F6D352C3F20001C1F2DF
:10151000620201240968A1FB0212A11E01EB9211D3
:101520000A0E18D14EF21002F023CEF200025160E2
:1015300002F613510B700021916007210F281160F2
:1015400009D8A01E0F2100F003FD40F22810C3F2BD
:0A155000000004700024204610BDC6
:10155A0040F200104FF65F71C3F20000C0F20301BF
:10156A000068C16040F22411C3F200010A68C3682E
:10157A009B0606D40B689B1AB3F57A7FF7D903202A
:06158A00704700207047CD
:1015900010B582B044F60C01C5F6020108680A686D
:1015A000400740F22410C3F200000DD5022363F37C
:1015B00002020A60026851F8083C9B0404D40368E4
:1015C0009B1AB3F57A7FF6D900220192CA680223EA
:1015D00063F38F32CA60CA6802F440420192019AF2
:1015E000CA689204FCD544F20044C5F60204D4F85B
:1015F000001441F48071C4F80014216F21F0180127
:101600002167216901F03802A16A102A07D0182A3F
:1016100040F0F38001F00301022940F0EE802168E0
:10162000D4F8001441F48071C4F800140168D4F8AF
:101630000024D20504D40268521A642AF7D931E191
:10164000216F41F2883241F0010121670168236F67
:101650009B0704D403685B1A9342F8D922E12169FD
:1016600001F03801182940F0D680A16A40F2F33227
:1016700011405229216B40F015810A466FF35F2219
:10168000272A40F00F8101F47E42B2F5007F40F03E
:10169000098101F4FE02B2F5803F40F0038101F0C0
:1016A000FE41B1F1807F40F0FD80616B4FF6F87232
:1016B000114210D0E16A21F00101E1620168026883
:1016C0008A42FCD0616B4FF6F87291436163E16A24
:1016D00041F00101E16242F2000CC5F2002CDCF89D
:1016E000002012070DD1DCF80020012363F3030270
:1016F000CCF80020DCF8002002F00F02012A40F0B4
:10170000D280A269E269E269226AA269A26922F42E
:101710007062A2612268920140F1C58022690323B0
:1017200063F302022261026841F28833216901F009
:101730003801182904D00168891A9942F6D9B2E013
:10174000A06900071EBFA06920F00F00A061DCF8AF
:10175000000010F00E0F0DD0DCF80000012161F345
:101760000300CCF80000DCF8000000F00F000128B6
:1017700040F09980A06910F0700F1EBFA06920F0A2
:101780007000A061E06910F0700F1EBFE06920F0EA
:101790007000E061E06910F4E06F1EBFE06920F4C2
:1017A000E060E061206A10F0700F1EBF206A20F038
:1017B00070002062FEF78AFFA16942F23852C0F63B
:1017C0000002C1F30321515C40F22812C3F200026F
:1017D000A36940F22C1301F01F011278C3F2000339
:1017E00020FA01F11020002A196018BF0F20FFF71E
:1017F00087FE002857D102B010BD216841F4803126
:1018000021600168226892033FF50AAF0268521A0C
:10181000642AF7D946E0216821F0807121600168CF
:101820002268920104D50268521A022AF8D939E0D6
:10183000A16A40F2F33291434FF6F8725231A1623D
:1018400040F22721C0F201112163E16A21F0010178
:10185000E162616B91436163E16A022262F3830199
:10186000E162E16A21F00201E162E16A41F4803162
:10187000E162E16A41F40031E162E16A41F4802110
:10188000E162E16A41F00101E162216841F08071A9
:1018900021600168226892013FF51DAF0268521A6B
:0818A000022AF7D972B672B6F4
:1018A80040F22410C3F20000016801310160704762
:1018B8002DE9F04782B00020019040F22C1040F250
:1018C8008804C3F20000C3F2000448F2B51240F2E3
:1018D8006F480168C1F64E32A56DC4F2020820684F
:1018E800A1FB021A40452F68296808DCA8F5747125
:1018F800884211DC4839884225DC473924E045F222
:101908002F42C5F60202904214DC08F148029042C8
:101918003BDCA2F1470117E001F56271884212DC55
:10192800A1F28731884218D01831884215D001F5C4
:1019380056710FE03C329042D4BF3B3A013290429C
:1019480030D0143228E00131884206D0183188425C
:1019580003D01831884240F09881E16D082201F0E7
:101968001F01A8F160098A403A4267D0042348451C
:1019780006DCA8F58066B042D4BF303E303647E07A
:10198800404543DCA8F1300642E001329042E4D001
:1019980045F20842C5F60202904203D01432904242
:1019A80040F073810268E36D03F01F0304279F4032
:1019B8000F4218BF12F004061CD102279F400F42A5
:1019C80018BF12F0020640F0B780D940090740F16D
:1019D8005C8112F0080100F05881016821F00E01C5
:1019E8000160012000FA03F16960606584F8350040
:1019F800E16C00E111046F6000F1B080910600F124
:101A0800B180016821F004010160ABE008F1300603
:101A1800B042CCBF01362F3EB04203D01836B04298
:101A280018BF082306681E4208D0036823F0040381
:101A38000360AA60626D42F00102626501228A4079
:101A48003A4221D0484506DCA8F580639842D4BFC5
:101A5800303B303306E0404502DCA8F1300301E0BA
:101A680008F130039842D4BF2F3B0133984203D08A
:101A78001833984240F0128143691B0604D5AA60C6
:101A8800626D42F00202626504228A403A4221D025
:101A9800484506DCA8F580639842D4BF303B303314
:101AA80006E0404502DCA8F1300301E008F130030C
:101AB8009842D4BF2F3B0133984203D01833984241
:101AC80040F0EE8003689B0704D5AA60626D42F07F
:101AD8000402626510228A403A424CD008234845E5
:101AE80006DCA8F58066B042D4BF303E303606E04A
:101AF800404502DCA8F1300601E008F13006B042AA
:101B0800CCBF01362F3EB04203D01836B04218BFC2
:101B1800042306681E422ED0AA6002685203026897
:101B280006D4D20506D4026822F00802026001E059
:101B3800100319D4226C18E011046F6000F1A8801A
:101B4800910600F1A980016821F00A0101600120D5
:101B580084F83500002084F834009DE0D00301D4D7
:101B6800A16C89E0216C87E0A26C22B120469047E5
:101B7800E06D00F01F01202000FA01F23A425AD02D
:101B880020681023484506DCA8F58067B842D4BF12
:101B9800303F303706E0404502DCA8F1300701E06D
:101BA80008F13007B842CCBF01372F3FB84203D005
:101BB8001837B84218BF022307681F423BD0AA60F3
:101BC80094F83520042A02681AD122F0160202601D
:101BD800426922F080024261226CA36C1A4303D04E
:101BE800026822F0080202603F208840A8600120B5
:101BF80084F83500216D002084F83400E9BB44E006
:101C0800510301680CD4C9050ED4016821F01001F4
:101C18000160012084F83500002084F8340003E0D6
:101C2800080301D4616C00E0E16B21B140F2880047
:101C3800C3F200008847606D38B3606DC0071AD0E2
:101C4800042084F835002068016821F00101016052
:101C5800019901310191B1EB9A2F02D80168C907A6
:101C6800F6D10068C00714BF0320012084F83500AE
:101C7800002084F83400E16C39B140F28800C3F2E6
:101C8800000002B0BDE8F047084702B0BDE8F087A1
:101C9800D00301D4616CEFE7E16BEDE70268F3E68E
:041CA800026817E7D0
:101CAC0081B044F2D840C5F60200016841F0010150
:101CBC0001600068002100F00100009000984EF6D1
:101CCC000C50CEF2000000684EF20B40CEF2000039
:101CDC0001704EF20010CEF200004FF40061016072
:041CEC0001B070478C
:101CF0002DE9D04187B044F2E0400024C5F602004F
:101D0000A046CDE904440168C5F6020841F010017F
:101D100001600168032701F010010091009901683A
:101D200041F004010160016801F004010091009993
:101D3000016841F020010160016801F0200100917B
:101D40000099016841F080010160016801F08001A3
:101D500000910099016841F001010160016801F002
:101D6000010100910099016841F0020101600168E0
:101D700001F0020100910099016841F04001016009
:101D8000016801F0400100910099016841F00801EB
:101D90000160006801A900F0080000900098039419
:101DA0004AF2FF70CDE9010708F5805000F0D6FA3D
:101DB00043F6FF7001A9CDE9010708F5006003941F
:101DC00000F0CCFA08F5A05001A94FF6FF76039475
:101DD000CDE9016700F0C2FA404601A9CDE90167EB
:101DE000039400F0BBFA08F5806001A9CDE9016712
:101DF000039400F0B3FA08F5C05001A9CDE90167DA
:101E0000039400F0ABFA08F5406001A9CDE9016741
:0C1E1000039400F0A3FA07B0BDE8D081F5
:101E1C00E0B5AEB040F2041544F20806C3F200057A
:101E2C00C5F600067F21A6F108000027696045E988
:101E3C000107FF21AF61C5E90217C5E90477697F86
:101E4C00D1B902A8B0212F77FFF7E4F84FF4800046
:101E5C00CDE900074FF480702C906846FEF7B6FC75
:101E6C00002867D144F27040C5F60200016841F4C5
:101E7C000041016055F8040C02216977C168C9065C
:101E8C0054D4CA21416253214162C168490616D417
:101E9C00F943C16040F22411C3F200010A68C3681F
:101EAC005B060CD40B689B1AB3F57A7FF7D9032128
:101EBC006977C06855F8040CFF21416272B68168DD
:101ECC0021F4E00121F04001816095E88E00394356
:101EDC006F69394387683943816043EA0241016184
:101EEC00706820F0800070603068800605D4FFF7C1
:101EFC002EFB68B103206877DCE7306820F0200007
:101F0C003060FFF724FBB0B9306840F0200030603F
:101F1C0055F8040C2969AA69C36C114323F0030317
:101F2C00C364C26C1143C164FF2141620120687714
:101F3C002EB0E0BD72B603206877306840F0200008
:041F4C003060B7E763
:101F500000B54EF60C5C4FF0FF3ECEF2000CDCF804
:101F60000030C3F3022383F00702042A28BF0422AF
:101F70000EFA02F29143033B00F00F0228BF994092
:101F800000F16043043A03F56443624400284FEAD9
:0C1F9000011048BF02F10C03187000BDE6
:101F9C002DE9F04744F2004200F10807C5F60202B1
:101FAC00D0F81CC0D0E9004A97E88043936A03F04C
:101FBC000303032B04BF0120BDE8F087136823F053
:101FCC008063136040F22413C3F200031D6816688B
:101FDC00360104D51E68761B022EF8D952E0956A9C
:101FEC004FF4FE0625F47C3506EB084645EA04342E
:101FFC0094624FF47E44AAF1010504EB472406F4E5
:10200C00FE066FF35F2515FA84F44FF0FE4505EBE1
:10201C00096505F0FE452C4434449463D46A24F0DD
:10202C00C00444EA0E07D762D76A806927F02007FC
:10203C003843D062D06A4FF6F87720F01000D062A7
:10204C00D06BB843012940EACC00D063D06A40F091
:10205C001000D0624FF4001008BF4FF4801000291C
:10206C00D16A08BF4FF400200843D062106840F0DA
:10207C008060106018681168090106D41968091A83
:10208C000329F8D30320BDE8F0870020BDE8F087D2
:10209C002DE9F04744F2004200F10807C5F60202B0
:1020AC00D0F81CC0D0E9004A97E88043936A03F04B
:1020BC000303032B04BF0120BDE8F087136823F052
:1020CC008053136040F22413C3F200031D6816689A
:1020DC00B60004D51E68761B022EF8D952E0956A1C
:1020EC004FF4FE0625F07C7506EB084645EA0454D1
:1020FC0094624FF47E44AAF1010504EB472406F4E4
:10210C00FE066FF35F2515FA84F44FF0FE4505EBE0
:10211C00096505F0FE452C4434441464D46A24F457
:10212C00406444EA0E07D762D76A806927F40077C7
:10213C003843D062D06A4FF6F87720F48070D062C2
:10214C00506CB843012940EACC005064D06A40F48A
:10215C008070D0624FF0807008BF4FF400000029EF
:10216C00D16A08BF4FF480000843D062106840F079
:10217C008050106018681168890006D41968091A13
:10218C000329F8D30320BDE8F0870020BDE8F087D1
:10219C0090F83510022916D180B540F20F42016833
:1021AC00C4F20202914212DCA2F5687C61451DDC8E
:1021BC00A2F5747C61452FDCA2F2FF3C614548D04E
:1021CC00A2F2E73C43E080214165012163E002F18A
:1021DC00600C614515DC02F1300C614523DC02F129
:1021EC00010C614535D002F1190C30E0A2F55C7C94
:1021FC0061451FDCA2F29F3C61452AD0A2F2873CCC
:10220C0025E002F1900C61451BDC02F1610C61458B
:10221C001FD002F1790C1AE0A2F2CF3C614518D024
:10222C00A2F2B73C13E002F1310C614511D002F17E
:10223C00490C0CE0A2F26F3C61450AD0A2F2573C6B
:10224C0005E002F1A90C614503D002F1910C614546
:10225C0028D191424FF0040280F8352006DC6F2023
:10226C00C4F20200814207DD303006E040F26F40DC
:10227C00C4F20200814203DC3038814203DD03E00A
:10228C003030814209DC2F38086820F001000860EA
:10229C000021BDE80840084670471930814218BF3C
:1022AC001838F1E70A6822F00E020A6045F257422C
:1022BC00C5F6020291420A6822F001020A6007DCAC
:1022CC0045F22F42C5F60202914207DD013206E0CB
:1022DC0045F27F42C5F60202914204DC273A914254
:1022EC0007D0143203E01532914202D0143A9142D5
:1022FC0019D1D0E91813D0E916EC0A6822F48072CF
:10230C000A600CF01F01012202FA01F1CEF8041050
:10231C00816E5960C16E31B10A6822F480720A6014
:10232C00D0E91C124A60012180F83510026D0021A1
:0C233C00002A80F83410ACD09047A9E7CC
:10234800806B0021A0F86A10A0F86210012180F8C3
:042358008110704739
:10235C002DE9F04F85B00A680290002A00F0D78072
:10236C0000F1264342F200488E4603F1FF77C5F692
:10237C0002080A214FEAB723404508BF092100246F
:10238C00082B38BF4FEAB7214FF001080027002671
:10239C000091CDF80CE0A8F1010A012000FA0AFC2A
:1023AC001CEA020900F0A880DEF804B071460BF0BC
:1023BC00030EAEF10102012A18D8700001900298A8
:1023CC000322CD68BA408368BD4093432B4383609E
:1023DC00D5434268CBF3001322EA0C02AC46054607
:1023EC0003FA0AF301981A436A600CE0BEF1030F7A
:1023FC0001D1029D2AE0032000FA07F138466FEA6A
:10240C00010CDDE902518A68EB6803EA0C0302FA5D
:10241C0000F11943BEF1020FE96017D16FF0030010
:10242C0004F01C0300EA5A01039829440F22D0F847
:10243C0010C09A400D6A0CFA03F325EA0202029DC1
:10244C001A430A62D0F804B00BF0030E032029687B
:10245C0000FA07F291430EFA07F211431BF4403FC6
:10246C002960DDF80CE047D044F2F44040F2084C0F
:10247C00C5F60200C5F6000C016841F002010160CE
:10248C0001680F2001F0020104912AF00301049A63
:10249C0004F00C0251F80C3000FA02F50098AB4332
:1024AC0000FA02F24FF0B0401A4341F80C200168D8
:1024BC00DEF8042041EA0903D50258BF21EA0903DA
:1024CC00036004309502016841EA090358BF21EA10
:1024DC00090303609503D0F8801041EA090358BF43
:1024EC0021EA0903C0F88030D203C16F41EA090325
:1024FC0058BF21EA0903C367DEF800200136023712
:10250C00043432FA08F108F101087FF444AF05B045
:04251C00BDE8F08F97
:10252000FEF762FF4EF68850CEF20000016851F4CB
:0825300070010160FEF76AFD75
:10253800000000000000000001020304060708096B
:102548006D25000800000030290100007F250008E3
:102558002C0100306825000804000000171000084E
:042568000090D0030C
:10256C00206861680834002200E042540139FCD52F
:02257C007047A6
:10257E0020686168A2680C3401E08B5C8354013AD8
:04258E00FBD57047C2
:0400000508002521A9
:00000001FF
